:020000020000FC
:100000000FC0A9C0B3C0B5C0B5C0B5C0B0C0B0C006
:04001000B4C0B2C006
:10002000F89400E810E006BD16BD0AE208BB09E03E
:1000300007BBB0E0A0E6D0E0C0EA00E00D93BD173A
:10004000E9F7AC17D9F70EE90DBF00E60ABF0EE0DD
:1000500008BF00E005BD00E105BF01E80FBD02E0FB
:1000600003BF00E006BF00E009BD00E008BD00E6F8
:1000700007B900E003B907E006B904E104BB00E8F2
:1000800008B909E319E301BD11BD00E005BB00E4B7
:100090000BBF00E009BF04E1202E05E0302EB0E0E8
:1000A000A0E0789404B700FF04C00E7F04BF91E085
:1000B00000C001E0902790FF30C0B0E0A0E000E277
:1000C00007B902E36DD002E059D0102F0FEF011BEA
:1000D000D0E0C02F10E002E3C00FD11F00E607B947
:1000E00002E35ED0A89501E049D0023B18F43A94AF
:1000F00019F413C005E0302ECA1BDB0B08F40DC049
:10010000022D003F18F40AE0200E02C00FEF202E4F
:1001100026BE11960AE044D0D2CF00E006BF0AE026
:100120003FD0C39800E003BF00E006B900E007B984
:1001300000E808B903E005BD00E40BBF09E311E3E3
:1001400001BD11BD90E003E012E020E300BF10BF4D
:1001500025BF8895FFCFFFB60F9300E006BF02E3EF
:100160001FD0A89506B301FFFCCF5ACF189518955C
:100170001895189518951895189518951F9310E0CF
:1001800016B917B11C7F102B17B900E003B907ECA3
:1001900006B906B106FDFDCF04B105B11F91089562
:1001A0001F932F932BE11BE31A95F1F72A95D9F7AB
:0A01B0000A95C1F72F911F910895E1
:00000001FF
